:1000000072C196C1A0C49FC493C192C191C190C155
:100010008FC18EC18DC151C48BC18AC189C188C1B4
:1000200087C100003900360000003A0037000000A8
:100030000000000403020100000102040810204037
:100040008004020100003B003800010101010101B0
:1000500001010202024446372D303031E694B9E8FE
:10006000A18C20777332383132E381AE3135E79598
:10007000AAE79BAEE381AEE4BFA1E58FB7E382922E
:10008000E980B2E8A18C42E4BFA1E58FB70044410A
:10009000362D303031E694B9E8A18C2077733238B0
:1000A0003132E381AE3130E795AAE79BAEE381AE12
:1000B000E4BFA1E58FB7E38292E6B89BE9809FE4B5
:1000C000BFA1E58FB7004437352D303031E694B904
:1000D000E8A18C20777332383132E381AE37E7956F
:1000E000AAE79BAEE381AEE4BFA1E58FB7E38292BE
:1000F000E6B3A8E6848F42E4BFA1E58FB70044339E
:10010000342D303031E694B9E8A18C207773323841
:100110003132E381AE33E795AAE79BAEE381AEE4EB
:10012000BFA1E58FB7E38292E5819CE6ADA242E4F0
:10013000BFA1E58FB7004432332D303031E694B99A
:10014000E8A18C20777332383132E381AE32E79503
:10015000AAE79BAEE381AEE4BFA1E58FB7E382924D
:10016000E980B2E8A18C41E4BFA1E58FB70044313A
:10017000322D303031E694B9E8A18C2077733238D3
:100180003132E381AE31E795AAE79BAEE381AEE47D
:10019000BFA1E58FB7E38292E6B3A8E6848F41E47E
:1001A000BFA1E58FB7004430312D303031E694B92E
:1001B000E8A18C20777332383132E381AE30E79595
:1001C000AAE79BAEE381AEE4BFA1E58FB7E38292DD
:1001D000E8ADA6E68892E4BFA1E58FB700443030D1
:1001E0002D303031E694B9E8A18C20777332383164
:1001F00032E381AE30E795AAE79BAEE381AEE4BF80
:10020000A1E58FB7E38292E5819CE6ADA241E4BF10
:10021000A1E58FB700532D303031E694B9E8A18CB9
:1002200020E78FBEE59CA8E381AEE382B9E3838635
:10023000E383BCE382BFE382B900E99D92E4BFA1FE
:10024000E58FB7E382B3E3839EE383B3E38389203F
:1002500047312D303031E694B9E8A18CE381A7E431
:10026000BFA1E58FB7E6A99FE38292E99D92E38162
:10027000AB00E9BB84E4BFA1E58FB7E382B3E383BE
:100280009EE383B3E383892059312D303031E694E6
:10029000B9E8A18CE381A7E4BFA1E58FB7E6A99FE8
:1002A000E38292E9BB84E381AB00E8B5A4E4BFA19B
:1002B000E58FB7E382B3E3839EE383B3E3838920CF
:1002C00052312D303031E694B9E8A18CE381A7E4B6
:1002D000BFA1E58FB7E6A99FE38292E8B5A4E381C9
:1002E000AB006808DD0811241FBECFE5D2E0DEBFF9
:1002F000CDBF21E0A4E9B0E001C01D92AB3CB20744
:10030000E1F710E0A0E6B0E0E2EBF2E102C0059018
:100310000D92A439B107D9F711E0C2E7D1E003C0CB
:100320002197FE01B4D7C137D107D1F784D3B5C720
:1003300067CE1D9887E087B9369A3699FECF84B18B
:1003400095B10895AF92BF92CF92DF92EF92FF9254
:100350000F931F93CF93DF936C017B018B01040FED
:10036000151FEB015E01AE18BF08C017D10759F089
:100370006991D601ED91FC910190F081E02DC601CB
:100380000995892B79F7C501DF91CF911F910F91C5
:10039000FF90EF90DF90CF90BF90AF90089590E0E6
:1003A000FC01E25DFF4F3491FC01E75CFF4F2491BB
:1003B000FC01E65BFF4FE491EE23B9F0332329F013
:1003C000323019F198F43130E1F0F0E0EE0FFF1F18
:1003D000EC5BFF4FA591B4918FB7F894EC9161114C
:1003E00017C020952E232C938FBF0895333029F00A
:1003F000343059F78FB58F7D02C08FB58F778FBDA1
:10040000E4CF80B78F7780BFE0CF80B78F7DFBCF01
:100410002E2BE9CFCF93DF9390E0FC01E75CFF4FF9
:100420002491865B9F4FFC0184918823C9F090E062
:10043000880F991FFC01E85DFF4FA591B491FC0165
:10044000EC5BFF4FC591D49161110DC09FB7F8943B
:100450008C91209582238C938881282328839FBFA9
:10046000DF91CF910895623051F49FB7F8943C9199
:10047000822F809583238C93E8812E2BEFCF8FB72B
:10048000F894EC912E2B2C938FBFEACF20919F01F3
:100490003091A0012817390771F490919D01809146
:1004A0009E01981741F0E0919D01F0E0EC5AFE4F5B
:1004B000808190E008958FEF9FEF08950895EF9267
:1004C000FF920F931F93CF93DF93DC015C96ED9027
:1004D000FC905D97E114F10479F481E090E01396CB
:1004E0009C938E93129790E080E0DF91CF911F91C3
:1004F0000F91FF90EF9008955196ED91FC915297D6
:1005000050968C915097982F90950FB75E962C919E
:100510005E97122F127021FD6095F89420811123AF
:1005200019F1282B2083E7012197F1F728E0462FC6
:1005300050E0308160FF1AC0382B3083E7012197EB
:10054000F1F7BA0175956795215089F7112381F06C
:100550008081892380830FBF5C968D919C91019748
:10056000F1F781E090E0C1CF2923DCCF3923E5CF3B
:100570009081892BEFCF20919F013091A001281706
:10058000390769F480919E0120919D0190E0805C83
:100590009F4F821B910960E470E052D6089590E06D
:1005A00080E0089520919F013091A001281739071C
:1005B000B9F490919D0180919E01981789F0E09186
:1005C0009D01F0E0EC5AFE4F808120919D0130E0CA
:1005D0002F5F3F4F2F73332720939D0190E00895A5
:1005E0008FEF9FEF089590E080E00895E091A301E0
:1005F000F091A40180819091A201892B8083808158
:100600009091A10189238083000000000000000078
:1006100000000000000000000895E091A301F091A7
:10062000A40180819091A201892B808300000000A9
:100630000000000000000000E091A301F091A4017F
:1006400080819091A101892380830895362F803481
:1006500050F490E063E070E0E2D5FC01EC56FF4F0F
:100660003083418322830895CF93C82F20E040E058
:1006700060E0ECDF20E040E060E081E08C0FE6DF4E
:1006800020E040E060E082E08C0FE0DF24E040E02A
:1006900068E183E08C0FCF91D9CFCF93C82F20E0B2
:1006A00040E460E1D3DF20E040E060E081E08C0FD7
:1006B000CDDF20E040E060E082E08C0FC7DF24E087
:1006C00040E068E183E08C0FCF91C0CFCF93C82F7B
:1006D00020E040E060E0BADF20E040E060E081E060
:1006E0008C0FB4DF20E040E460E182E08C0FAEDFED
:1006F00020E040E060E083E08C0FCF91A7CFCF9364
:10070000C82F20E040E060E0A1DF20E040E460E0AE
:1007100081E08C0F9BDF20E040E060E082E08C0F06
:1007200095DF20E040E060E083E08C0FCF918ECF3A
:10073000CF93C82F20E040E060E088DF20E040E079
:1007400060E081E08C0F82DF24E040E068E182E03D
:100750008C0F7CDF20E040E060E083E08C0FCF91E5
:1007600075CFCF93C82F20E040E060E06FDF20E03E
:1007700040E060E081E08C0F69DF20E040E060E075
:1007800082E08C0F63DF20E040E460E183E08C0FC7
:10079000CF915CCFCF93C82F20E040E460E156DFDB
:1007A00020E040E060E081E08C0F50DF20E040E09E
:1007B00060E082E08C0F4ADF20E040E460E183E00B
:1007C0008C0FCF9143CF0F931F93CF93F89404E9ED
:1007D00010E0F801C1918F01C7FF1FC01EDFC6FFE7
:1007E0001EC01BDFC5FF1DC018DFC4FF1CC015DF06
:1007F000C3FF1BC012DFC2FF1AC00FDFC1FF19C049
:100800000CDFC0FF18C009DFF1E004351F0709F74E
:100810007894CF911F910F910895E8DEE0CFE6DE46
:10082000E1CFE4DEE2CFE2DEE3CFE0DEE4CFDEDE06
:10083000E5CFDCDEE6CFDADEE7CFFC010190002079
:10084000E9F73197AF01481B590BBC018CEA91E0E5
:1008500079CD0F931F93CF93DF938C01D0E0C0E04D
:10086000F801EC0FFD1F6491662339F08CEA91E0EA
:1008700026DE892B11F02196F3CF42E050E06FE79E
:1008800070E08CEA91E05EDD8C0F9D1FDF91CF91CF
:100890001F910F910895CF93DF93C0E6D0E0688158
:1008A00082E090E0AED4698183E090E0AAD46A81CE
:1008B00084E090E0DF91CF91A4C41F920F920FB615
:1008C0000F9211242F933F938F939F93AF93BF93D6
:1008D0008091990190919A01A0919B01B0919C0106
:1008E0003091980125E5230F2D3728F028ED230FAF
:1008F0000196A11DB11D20939801809399019093B9
:100900009A01A0939B01B0939C01809194019091D6
:100910009501A0919601B09197010196A11DB11D7D
:100920008093940190939501A0939601B0939701C1
:10093000BF91AF919F918F913F912F910F900FBEDB
:100940000F901F9018951F920F920FB60F921124BF
:100950002F933F934F935F936F937F938F939F93C7
:10096000AF93BF93EF93FF93E0919F01F091A001AC
:10097000309749F0A685B7858585968D91FF14C07F
:100980009C918923A1F4FF91EF91BF91AF919F9129
:100990008F917F916F915F914F913F912F910F9028
:1009A0000FBE0F901F9018959C91892361F7A38922
:1009B000B4899C918589809589238C9386899789B0
:1009C0000197F1F7608D718DA685B785558538E063
:1009D00020E0CB010197F1F7822F90E09595879564
:1009E000282F4C91452309F02068315091F7868DCE
:1009F00081FD209580919E0190E001968F7399274B
:100A000030919D01381799F0A0919E01B0E0AC5A49
:100A1000BE4F2C9380939E01828D938D0197F1F7A9
:100A2000A389B4898C919589892B8C93ACCF868DC1
:100A30008160868FF1CFCF93DF93CDB7DEB72E974E
:100A40000FB6F894DEBF0FBECDBF789480B782603A
:100A500080BF80B7816080BF83B7826083BF83B768
:100A6000816083BF89B7816089BF1EBC8EB58260FB
:100A70008EBD8EB581608EBD8FB581608FBD329A7F
:100A8000319A309A379A61E080E0C4DC61E082E01C
:100A9000C1DC61E083E0BEDC61E088E0BBDC61E0FA
:100AA00084E0B8DC62E086E0B5DC61E085E0B2DCE1
:100AB00060E080E074DC60E082E071DC61E083E0B3
:100AC0006EDC60E088E06BDC60E084E068DC109263
:100AD000C7011092C6011092C5011092C401109274
:100AE000C3011092C2018DE990E09093C9018093F7
:100AF000C8019091B8019B30C8F52DE330E03093E8
:100B0000C3012093C2012BE930E03093C50120934B
:100B1000C4012CE630E03093C7012093C6018BB7A7
:100B200020E1983008F020E2822B8BBF22E330E0F6
:100B3000983030F020E430E09B3010F030E020E0DE
:100B40003093C0012093BF01492F50E0983008F046
:100B5000AEC181E001C0880F9A95EAF78093C10188
:100B60008091C8019091C9010197F1F78091C60168
:100B70009091C701892B49F1E0919F01F091A0016B
:100B800021E0EC3AF20709F1309739F0A389B489F2
:100B90009C918589809589238C938091CA018E7F51
:100BA0008093CA0110929E0110929D018CEA91E0FF
:100BB0009093A00180939F01E091BF01F091C0014B
:100BC00080819091C101892B808384E690E0A0E030
:100BD000B0E08093B0019093B101A093B201B093C3
:100BE000B30181E090E005D38093A50182E090E01D
:100BF00000D38093A6018091A5019091A6018A3A25
:100C0000910509F45EC18AEA90E09093A601809371
:100C1000A50181E090E0EDD28A3A21F06AEA81E014
:100C200090E0EFD21091A60182E090E0E2D2181796
:100C300021F0612F82E090E0E4D22DDE61E081E0DE
:100C4000E9DB60E081E0ABDBEBE4F0E0E491F0E0D5
:100C5000EE0FFF1FEC5BFF4F859194919093A401E1
:100C60008093A301EAE3F0E0E491E093A201E09530
:100C7000E093A1013FE7E32E33E0F32ECE0101968E
:100C80006C011E019EE0290E311C4CE2442E5524BD
:100C900053945BE4852E912C92E4692E8091AB01F4
:100CA000811113C0E1E0E093AB0129DD84E072DD46
:100CB00088E057DD8CE03CDD80E108DD84E1EDDC9F
:100CC00088E1D2DC8CE11BDD7EDD8EE1A82EB12C2B
:100CD00010E000E060E088E062DBC7010197F1F717
:100CE00028DB8D3C924014F00F5F1F4F61E088E0DD
:100CF00056DBC7010197F1F71CDB8C3C910514F41E
:100D00000F5F1F4F60E088E04ADBC7010197F1F7F2
:100D100010DB8D3C924014F00F5F1F4F60E088E0C5
:100D20003EDBC7010197F1F704DB8D3C924014F0E4
:100D30000F5F1F4F61E088E032DBC7010197F1F7D9
:100D4000F8DA8C3C910514F40F5F1F4F60E088E0E7
:100D500026DBC7010197F1F7ECDA8D3C924014F0E5
:100D60000F5F1F4F61E088E01ADBC7010197F1F7C1
:100D7000E0DA8C3C910514F40F5F1F4F61E088E0CE
:100D80000EDBC7010197F1F7D4DA8C3C910514F41E
:100D90000F5F1F4F21E0A21AB10809F09BCF053E5B
:100DA000110524F010926C0010926B0080916B0082
:100DB00090916C008C32914020F050926C004092E7
:100DC0006B0000916B0010916C000B34110508F062
:100DD00088C061E080E0E3DA60E082E0E0DA60E0D1
:100DE00083E0DDDAF2E5F09364000F5F1F4F1093AC
:100DF0006C0000936B00F6012EE011922A95E9F742
:100E00008CEA91E0B8DB181619060CF0EEC08601EA
:100E100056018CEA91E0C6DBF50181935F018D30CC
:100E200019F0E215F305A9F7609163005091620093
:100E3000409161003091600099E020E080E08130D5
:100E400009F477C008F46DC0823009F478C08330AB
:100E500009F47BC091500F5F1F4F9111F0CF2130EB
:100E600009F0C3C08981823509F075C08A81813358
:100E700009F0BBC010926C0010926B0061E084E03E
:100E80008EDA82E890E0D9DC44E050E060E670E081
:100E90008CEA91E057DA6DE08CEA91E010DB6AE0D1
:100EA0008CEA91E00CDB60E084E079DA9EC02AE015
:100EB00030E0241B350B81E001C0880F2A95EAF74A
:100EC0004DCE82E090E095D18093600083E090E089
:100ED00090D18093610084E090E08BD18093620098
:100EE000ADCE8091A9019091AA0160E00817190781
:100EF00060F480E054DA61E082E051DA60E083E09F
:100F00004EDA29E52093640070CF80E048DA60E093
:100F100082E045DA61E083E042DA87E480936400AE
:100F200064CF81E0F8017181731709F493CF80E0F9
:100F300091CFF80181818413FACF82E08BCFF80141
:100F400081818513F4CF83E085CFF8017181761319
:100F5000EECF21E07FCF893571F48A81813309F0AA
:100F600044C090926C0080926B0061E084E017DADC
:100F700086E890E088CF873489F48A818133A9F5A7
:100F80008091A7019091A80190936C0080936B00D1
:100F900061E084E004DA8AE890E075CF843409F0F7
:100FA00039C08A8190ED980F9A30A0F4792E770C91
:100FB000770CEB81E053E830B8F4F0E0EE51F84FF5
:100FC000872D099410C018C019C01AC01BC01CC0BE
:100FD0001DC01EC09FEB980F963018F48153782ED9
:100FE000E6CF6B82E6CF8BDBEEDB80E090E0892BF7
:100FF00009F454CE05D850CECDDBF6CFB2DBF4CF1A
:1010000097DBF2CF7CDBF0CF61DBEECF46DBECCFC2
:101010002BDBEACF833589F461E084E0C0D98EE828
:1010200090E00BDC80E990E008DC82E990E005DCF0
:1010300047E050E064E670E02BCF883441F561E092
:1010400084E0ADD98AEA92E004DC82E792E001DC38
:101050008AE392E0FEDB85E192E0FBDB8DED91E03F
:10106000F8DB86EA91E0F5DB8EE691E0F2DB86E3E1
:1010700091E0EFDB8EEF90E0ECDB86EC90E0E9DBDB
:101080008EE890E0E6DB85E590E0E3DB0CCF893489
:1010900009F0ABCF8A818D3209F0A7CF2B8180ED8B
:1010A000820F8A3008F0A1CF9C8180ED890F8A30B1
:1010B00008F09BCF8D8130ED380F3A3008F095CF96
:1010C000209361009093620080936300E4DB8DCFF6
:1010D0001092AF011092AE0188EE93E0A0E0B0E074
:1010E0008093B0019093B101A093B201B093B3018A
:1010F00081E790E09093AD018093AC011092C30121
:101100001092C2011092C5011092C4011092C70141
:101110001092C6011092C9011092C8016091CA01D3
:101120006E7F6D7F6093CA016695617081E068276C
:1011300085E035D961E085E06DD9EEE3F0E0E4913A
:10114000E093BC01EFE4F0E0E491F0E0EE0FFF1F6C
:10115000EC5BFF4F859194919093BE018093BD010C
:1011600060E086E057D98091CA0181FD03C061E04B
:1011700086E015D986E08093B801EFE3F0E0E491D2
:10118000E093B901E0E5F0E0E491F0E0EE0FFF1F3D
:10119000EE5DFF4F859194919093BB018093BA01CE
:1011A00086E990E09093AA018093A90181EE90E0F6
:1011B0009093A8018093A701089581E790E0909310
:1011C000AD018093AC0180919F019091A0018C5A58
:1011D000914071F4E091BF01F091C0019081809144
:1011E000C1018095892380831092A00110929F01F4
:1011F0000895E199FECF9FBB8EBBE09A99278DB3EE
:101200000895262FE199FECF1CBA9FBB8EBB2DBB44
:101210000FB6F894E29AE19A0FBE01960895002461
:10122000552704C0080E591F880F991F009729F0F1
:1012300076956795B8F37105B9F7802D952F0895C8
:1012400097FB072E16F4009406D077FD08D00BD03C
:1012500007FC05D03EF4909581959F4F08957095B9
:1012600061957F4F0895AA1BBB1B51E107C0AA1FC0
:10127000BB1FA617B70710F0A61BB70B881F991F37
:101280005A95A9F780959095BC01CD010895EE0F70
:10129000FF1F0590F491E02D099411E0C2E7D1E021
:1012A00003C0FE01F4DF2196C337D107D1F7F894CC
:0212B000FFCF6E
:1012B2002D303031472D722D3030312C010000009D
:1012C200005F02A201F3025E02BB02D20246020DDD
:1012D2000A00522D7200592D7200472D72004D00E6
:0412E20032002D00A9
:00000001FF
